:020000040000FA
:0600000041EF01F01200C7
:060008003AEF00F01200C7
:02002A000000D4
:0C007400DACFE4FFE2CFDAFFE9CFE4FFCF
:10008000EACFE4FFE652D9CFE6FFE1CFD9FF020E77
:10009000E126F350DF6E010EF4CFDBFF9EB08090BF
:1000A000A1A213D0A192AF0EE66E3C0EE66E15EC47
:1000B00001F0E552E5528080EF0EE66ED80EE66E56
:1000C0002BEC01F0E552E5529E90DF50F36E010EED
:1000D000DB50F46ED9CFE1FFE552E7CFD9FFE5520F
:1000E000E5CFEAFFE5CFE9FFE5CFDAFF1100850EA6
:1000F000E66EFAEC00F0E552A00EE66EDDEC00F0E4
:10010000E552AF0EE66E3C0EE66E15EC01F0E552E0
:0C011000E552F28EF28C9290FFD71200A4
:04011C002A0EF66E43
:10012000000EF76E000EF86E00010900F550856FA5
:100130000900F550866F03E1856701D03DD00900C5
:10014000F550806F0900F550816F0900F550826FFE
:1001500009000900F550E96E0900F550EA6E090042
:1001600009000900F550836F0900F550846F0900FC
:100170000900F6CF87F0F7CF88F0F8CF89F080C07C
:10018000F6FF81C0F7FF82C0F8FF0001835302E150
:10019000845307E00900F550EE6E8307F8E2840708
:1001A000F9D787C0F6FF88C0F7FF89C0F8FF0001C4
:0A01B0008507000E865BBFD7120022
:0601BA00D9CFE6FFE1CF02
:1001C000D9FFFE0EDB507E0BB16EB36AB26AA1920C
:1001D000FE0EDBAE02D0A08201D0A092DBB2CD86B3
:1001E000DBA002D0B18E01D0B19EB180E552E7CF45
:0401F000D9FF120021
:0C01F400D9CFE6FFE1CFD9FFFE0EDB50B3
:100200007E0BCD6EFE0EDBAC02D0CD8E01D0CD9E2E
:10021000CF6ACE6A9E90DBAE02D09D8001D09D90C9
:0A022000CD80E552E7CFD9FF1200B0
:06022A00D9CFE6FFE1CF91
:10023000D9FF020EE126FD0EDBCFDEFFDBCFDDFFB7
:10024000010EDB50B36EDF50B26ED9CFE1FFE55245
:06025000E7CFD9FF120008
:0A025600D9CFE6FFE1CFD9FF020E79
:10026000E126FD0EDBCFDEFFDBCFDDFF010EDB5035
:10027000CF6EDF50CE6ED9CFE1FFE552E7CFD9FF89
:0202800012006A
:0E02820015EE00F025EE00F0F86A019CA68E45
:0E029000A69C8EEC00F077EC00F0FDD712007B
:020000040030CA
:0E000000FF260E0EFF0180FF0FC00FE00F4025
:00000001FF
